:1000000023C032C031C030C02FC02EC0B3C02CC0FE
:100010002BC02AC029C028C027C026C025C024C0A4
:1000200023C022C021C03F065B4F666D7D077F6FF6
:10003000777C39585E79717674300E383F5C73671F
:10004000506D783E1C6E630011241FBECFE5D4E0D6
:10005000DEBFCDBF20E0A0E6B0E001C01D92AE360D
:10006000B207E1F7CCD098C2CBCF882311F0C09A69
:100070000895C098089581312EE0920708F463C076
:100080009C01A9E8B8E852D2AC0156954795529523
:1000900042954F7045275F7045279A0147D2969544
:1000A0008795929582958F7089279F708927982FC1
:1000B0002CE3829F4019112403C0109262000DC0EE
:1000C000EDEC9E9FE12D1124E695E695E695F0E096
:1000D000EA5DFF4FE491E09362008DEC989F812DE3
:1000E0001124869586958695880F282F220F220F3A
:1000F000820F981BE92FF0E0EA5DFF4FE491E09357
:100100006300EDEC4E9FE12D1124E695E695E69512
:10011000F0E0EA5DFF4FE491E09364008DEC489FCE
:10012000812D1124869586958695880F982F990F95
:10013000990F890F481BE42FF0E0EA5DFF4FE4912F
:10014000E093650008956CE370E0DCD1962F482FB2
:100150006A3008F4B2CFB4CF882331F0E3E6F0E0A0
:100160008081806880830895E3E6F0E080818F7766
:10017000808308951F920F920FB60F9211242F9330
:100180003F934F935F936F937F938F939F93AF931F
:10019000BF93EF93FF938AB59BB58E519B4F9BBD49
:1001A0008ABD809166008F5F809366008436B0F0D0
:1001B00080916B0090916C00892B29F410926D0056
:1001C00080E053DFC59880916B0090916C0001979F
:1001D00090936C0080936B0010926600FF91EF91FA
:1001E000BF91AF919F918F917F916F915F914F914F
:1001F0003F912F910F900FBE0F901F901895CF93A6
:10020000DF9300D01F92CDB7DEB78FEF81BB87BBE6
:1002100014BA8CE385BB1FBC83E08EBD80E189BF2F
:10022000789480E022DFC59880E090E024DF80E0D1
:1002300090E088D1909361008093600001978835A9
:10024000924030F08AE090E09093610080936000EB
:100250000F2EF7E66F2EF0E07F2EF02D0F2EF8E632
:100260004F2EF0E05F2EF02D0F2EF9E62F2EF0E04E
:100270003F2EF02D01E010E00F2EF2E6AF2EF0E061
:10028000BF2EF02D0F2EF3E6CF2EF0E0DF2EF02D57
:100290000F2EF4E6EF2EF0E0FF2EF02D0F2EF5E6F8
:1002A0008F2EF0E09F2EF02D09839A991CC0F30148
:1002B00080818F3FD1F080818F5F8083808180310A
:1002C000A1F480916D00811110C080916000909127
:1002D00061008835F2E09F0740F401969093610039
:1002E0008093600002C0F30110829B991AC0F20152
:1002F00080818F3FC1F080818F5F808380818031DA
:1003000091F480916D0081110EC0809160009091F8
:100310006100009741F00197909361008093600025
:1003200002C0F20110829C992AC0F10180818F3FA6
:1003300041F180818F5F80838081803111F58091D0
:100340006D0081111EC0609160007091610080E0BD
:1003500090E0FDD020916000309161004CE3429F1D
:10036000C001439F900D112490936C0080936B000B
:1003700081E07BDEC59A81E080936D0002C0F101CF
:1003800010829D9916C080916A008F3FA1F0EAE625
:10039000F0E080818F5F80838081803161F4809183
:1003A0006D00813041F410926D0080E05EDEC598F2
:1003B00002C010926A0080916D008111A0C0F3010B
:1003C00080818F3F89F48091600090916100883531
:1003D000F2E09F0748F401969093610080936000DB
:1003E0008CEDF30180838BC0F20180818F3F09F097
:1003F00086C08091600090916100009709F47FC0F1
:10040000019790936100809360008CED808377C0AA
:10041000C8010A8002C0880F991F0A94E2F728B326
:10042000F5013081382311F0226001C02D7FF601E3
:100430003081382311F0246001C02B7FF701308117
:10044000382311F0286001C0277FF4013081382360
:1004500011F0206101C02F7E18BA809582BB28BBA5
:1004600080916D008130A9F580916B0090916C00B6
:1004700002DE9091660081E0923308F080E06CDE4D
:1004800080916B0090916C004E97A8F4809166006B
:10049000893158F080916600833348F0909166006E
:1004A00089819B3428F080E003C081E001C080E0B6
:1004B0008170DBDD15C080916B0090916C00CC9752
:1004C00078F49091660081E09B3408F080E0CDDD07
:1004D00007C08091600090916100CDDD81E03CDE3D
:1004E00087EE93E00197F1F700C00000EA81FB81FD
:1004F0003196FB83EA83389709F08ACFD6CE1B82E8
:100500001A8286CFAA1BBB1B51E107C0AA1FBB1FC3
:10051000A617B70710F0A61BB70B881F991F5A958F
:10052000A9F780959095BC01CD010895A29FB001D7
:10053000B39FC001A39F01D0B29F700D811D1124F4
:10054000911D0895A8E1B0E042E050E006C0019698
:10055000272F12D010C0DC01CB01FC01E199FECFA6
:1005600006C0FFBBEEBBE09A31960DB20D92415032
:100570005040B8F70895262FE199FECF9FBB8EBB60
:10058000E09A01970DB2021631F02DBB0FB6F89428
:0C059000E29AE19A0FBE0895F894FFCFA4
:00000001FF
